S00F0000746573746C63642E7372656322
S113000045C0000058C0000056C0000054C00000A5
S113001052C0000050C000004EC000004CC00000A0
S11300204AC0000048C0000046C0000044C00000B0
S113003042C0000040C000003EC000003CC00000C0
S11300403AC0000038C0000036C0000034C00000D0
S113005032C0000030C000002EC000002CC00000E0
S11300602AC0000028C0000026C0000024C00000F0
S113007022C0000020C000001EC000001CC0000000
S11300801AC0000018C0000016C0000011241FBED2
S1130090CFEFD0E1DEBFCDBF11E0A0E0B1E0EEECE8
S11300A0F1E000E00BBF02C007900D92AE30B10743
S11300B0D9F775D08AC0A4CF20E030E008C0EFECB7
S11300C0F7E03197F1F700C000002F5F3F4F28178A
S11300D03907ACF308958BB380648BBB8FEC97E046
S11300E00197F1F700C000008BB38F7B8BBB8FECC3
S11300F097E00197F1F700C000000895CF938FEFC8
S113010081BB8ABB15BA1BBAC0E2C5BBE4DFC5BB61
S1130110E2DF80E885BBDFDF15BADDDF80EF85BB7A
S1130120DADF15BAD8DF80E685BBD5DFCF91089535
S1130130CF93C82F85BB8BB380618BBBCCDFC295BB
S1130140C07FC5BB8BB380618BBBC5DFCF910895E6
S1130150CF93DF93EC0102C0EBDF219688818111FC
S1130160FBCFDF91CF910895CF93C82F85BB8BB37D
S11301708F7E8BBBB0DFC295C07FC5BB8BB38F7E38
S11301808BBBA9DFCF91089581E0EEDF8FE99FE07B
S11301900197F1F700C0000080E8E6CF08958FEFE3
S11301A084BB85BBABDF8FE19EE40197F1F700C010
S11301B00000EADF80E091E0CBDF95B381E089279E
S11101C085BB8AEF90E078DFF8CFF894FFCF8C
S11101CE48656C6C6F20776F726C64210000C2
S9030000FC
